:10000000B428A00088200C080D040319AF28A920EB
:1000100084132008800664000D280E288C0A03191A
:100020008D0F0B288006AF2823088C0021088D0037
:1000300001308E008F0164003C20031C2F288E0BA2
:100040001B28FF308F0703181B288C07031C8D0704
:10005000031CAF2832308E0000308F001B286D202B
:1000600008308F006E203C208E0C36288F0B3228F3
:100070006E2003140E08080022088400200884174C
:100080008004841300051F192006FF3E080092001B
:10009000220884000930930003105320920C930B24
:1000A0004D280314532884139F1D62280008200440
:1000B0001F1D20068000841700082004031C200652
:1000C00080006E2800082004031C20061F1920064B
:1000D00080008417200980056E281F171F0D063920
:1000E0008C007C208D008C0A7C201F1F8D281F1304
:1000F0008C000230A4208D2800308A000C08820772
:10010000013475340334153400343C340C34D934A0
:10011000FF3A84178005AF288D01E83E8C008D09D9
:10012000FC30031C96288C07031893288C07640066
:100130008D0F93280C189C288C1CA0280000A02848
:10014000080003108D0C8C0CFF3E0318A1280C082E
:10015000AF288C098D098C0A03198D0A08008313B6
:100160000313831264000800831686010D30850096
:1001700083120610831606108312861083168610CB
:1001800083120611831606118312861183168611B7
:1001900083120612831606128312861283168612A3
:1001A000831206138316061383128613831686138F
:1001B000831205168316051283127F30A6006F3056
:1001C000A7009030A8004130A9007F30AA007F30FE
:1001D000AB007F30AC007F30AD000530A2000130B5
:1001E000A00004309F000730A300A1011420031CCD
:1001F0003E29FF3C031DF6281420031C3E29AE00B7
:100200001420031C3E29A4000530A2000230A000E7
:1002100004309F002E0847202408472064002E0841
:10022000003C031D15292408A60064002E08013C8B
:10023000031D1F292408A7002708FE3CA80064000E
:100240002E08023C031D26292408A90064002E085C
:10025000033C031D30292408AA002A08FE3CAB00F9
:1002600064002E08043C031D37292408AC006400F8
:100270002E08053C031D3E292408AD0026088C00ED
:100280008D01063084000130012027088C008D018B
:10029000063084000230012028088C008D010630D1
:1002A00084000430012029088C008D010630840070
:1002B000083001202A088C008D010630840010309F
:1002C00001202B088C008D01063084002030012095
:1002D0002C088C008D0106308400403001202D0850
:0E02E0008C008D010630840080300120ED2856
:02400E00F53F7C
:00000001FF
